:04000000B401DD2842
:0800080008000408A70089109C
:100010000910091083168910091009100F3088057E
:1000200083122708B41832283A30A1009830912062
:100030003330A60046201330A1008830912046209E
:10004000643090204620643090202230A600462064
:10005000283031200C30312006303120B4142708EC
:1000600032283414A600341C40280910033C031C19
:10007000452845200730A100D03091200314080006
:100080003414FE3C0319D8280914341C3410891484
:100090000F3088052608F03988048910A60E341818
:1000A00046283230902003140800B513290803199C
:1000B000B5170530A8002730A30010306B2003309F
:1000C000A300E8306B20A30164306B20A3010A3049
:1000D0006B2024087228A2002508A1002408A00093
:1000E000B7202008A000A8030319B5132908031995
:1000F0007C282802031808002008031DB513B51B2F
:100100000800303ED328A301A200FF30A207031C41
:10011000A307031CD8280330A100DF3091208528D5
:10012000A101E83EA000A109FC30031C9A28A00709
:1001300003189728A0076400A10F97282018A0286B
:10014000A01CA4280000A4280800A2000530A800D4
:1001500023082102031DAE282208200204300318C0
:100160000130031902302805031DFF30D828A501EE
:10017000A4011030A600210DA40DA50D2208A40293
:100180002308031C230FA5020318CD282208A40767
:1001900023080318230FA5070310A00DA10DA60B1C
:1001A000BB282008D828840031088A003008820043
:1001B00083130313831264000800831607309F0023
:1001C0008312091183160911643083128A01832076
:1001D000BE01BA01BF01C0010130BC008316553019
:1001E00081008312A0308B008B178A110A12FD2820
:1001F0008B1B08008A110A124A2A8A01F8208601FC
:100200008A01F8208316F030860083128A01F820D4
:1002100064008A110A12861F022A8A01F8206400EB
:100220008A110A12061FD6298A01F82064008A1151
:100230000A12861E192A8A01F82064008A110A12FD
:10024000061EEC298A01F82064003C08013C8A1152
:100250000A12031DD2298A01F820FE308A010620E5
:1002600001308A0106208A01F8203E08BB008A017D
:10027000F8203E08A000A1010C30A200A3018A01D1
:10028000B7202408B2002508B3003208A0003308C4
:10029000A100A30100308A01A5208A110A12031DC2
:1002A00057298A01F8200C30BB078A01F8208A01FF
:1002B000F82064000C303E028A110A1203189429B7
:1002C0008A01F8200230A9003B08A400A5010530EE
:1002D000B000B1018A0155203A308A01062002306F
:1002E000A9003A08A400A5010530B000B1018A01B7
:1002F00055203A308A0106200230A9003F08A400A8
:10030000A5010530B000B1018A01552020308A01D5
:10031000062041308A0106204D308A0106208A01DC
:10032000F8208A110A12CD298A01F8200230A9008A
:10033000F4303B07B200FF300318013EB30032082F
:10034000A4003308A5000530B000B1018A01552092
:100350003A308A0106200230A9003A08A400A5011B
:100360000530B000B1018A0155203A308A010620DB
:100370000230A9003F08A400A5010530B000B1017A
:100380008A01552020308A01062050308A0106203B
:100390004D308A0106208A01F8208A01F820BC012C
:1003A0008A01F8208A01F8208A01FD288A01F820B4
:1003B000BA0A8A01F82064003C303A028A110A1213
:1003C000031CE7298A01F820BA018A01F8208A0172
:1003D000F8208A110A122B2A8A01F820BE0A8A0103
:1003E000F820640018303E028A110A12031CFD290D
:1003F0008A01F820BE018A01F8208A01F8208A11BA
:100400000A122B2A8A01F820BA038A01F820640014
:100410003C303A028A110A12031C142A8A01F8207D
:100420003B30BA008A01F8208A01F8208A110A12AA
:100430002B2A8A01F820BE038A01F82064001830B4
:100440003E028A110A12031C2B2A8A01F820173057
:10045000BE008A01F8208A01F8200130BD00640046
:100460001A303D028A110A120318422A8A01F82022
:100470000A308A0183208A01F820BD0A8A110A12F3
:10048000031D2F2A8A01F8200130BC008A01F820C0
:100490008A012229C00A64003D3040028A110A12F2
:1004A000031C702AC001BF0A64003C303F028A115D
:1004B0000A12031C6E2ABF01BA0A64003C303A02D9
:1004C0008A110A12031C6E2ABA01BE0A640018308F
:1004D0003E028A110A12031C6E2ABE010130BC00C2
:0A04E0000B11090063008A01722A63
:02400E00753DFE
:00000001FF
